:10000000180800104501000000000000000000007A
:10001000B1020000B1020000B102000000000000C7
:10002000000000000000000000000000B10200001D
:10003000B102000000000000B1020000B1020000A7
:10004000B1020000B1020000B1020000B1020000E4
:10005000B1020000B1020000B1020000B1020000D4
:10006000B1020000B1020000B1020000B1020000C4
:10007000B1020000B1020000B1020000B1020000B4
:10008000B1020000B1020000B1020000B1020000A4
:10009000B1020000B1020000B1020000B102000094
:1000A000B1020000B1020000B1020000B102000084
:1000B000B1020000B1020000B1020000B102000074
:1000C000B1020000F0B51A4F83B000F0BBF93868F8
:1000D0004FF4E13100F068FA164D174C00266969BB
:1000E000386841F480226A61144900F0F1F9002077
:1000F0000190019BA34205DC019A501C0190019BD9
:10010000A342F9DD69690E4821F480226A61314613
:1001100000F004FC0023019301990136A142DEDCCA
:10012000019A531C01930198A042F9DDD7E700BF63
:100130000C00001020C00920FFFF0F00EC0E000093
:10014000FC0E0000684620F007018D46F1B500F076
:10015000B1F84F484F49884235D04F4CA14232D276
:10016000024652F8046B0B46CD4343F8046B651905
:10017000A342C5F3810526D29DB1012D0BD0022DDE
:1001800005D0156800F108021D6001F1080352F85E
:10019000040B43F8040B52F8041B43F8041BA3425E
:1001A00011D296465EF8047B5668D568DEF80400E6
:1001B0009C464CF8047B5E60CCF80400DD60103394
:1001C0001032A342EDD335483549884234D0354CFE
:1001D000A14231D2024652F8046B0B46CD4343F89C
:1001E000046B6519A342C5F3810525D29DB1012D8C
:1001F0000BD0022D05D0156800F108021D6001F139
:10020000080352F8040B43F8040B52F8041B43F89C
:10021000041BA34210D294465CF8047B5668D56850
:10022000DCF80400194641F8047B5E604860DD603C
:1002300010331032A342EED31B491C48814221D215
:1002400000220B46CC4343F8042B04198342C4F329
:10025000810417D264B1012C06D0022C1CBF1A6095
:1002600001F1080343F8042B43F8042B834209D21D
:100270009E464EF8042B5A60CEF80420DA60103304
:100280008342F5D3FFF71EFFBDE8F1408546704776
:10029000340F0000000000100C000010340F0000AC
:1002A00000000010000000100C00001018000010EA
:1002B000FEE700BF3649202330B4C1F8A031D1F8A1
:1002C000A001334A10F0400FF9D0324D0124AA208A
:1002D00055230321C2F80411C2F80C411146C2F89B
:1002E0008450C2F88C00C2F88C30C2F88040C2F84A
:1002F0008C00C2F88C30D1F88830254A13F0806F1A
:10030000F9D00321AA245520C2F88010C2F88C40ED
:100310001146C2F88C00D1F888301D4A13F0407F96
:10032000F9D02324C2F8A440AA2055230124C2F8FE
:10033000AC001146C2F8AC30C2F8A040C2F8AC0024
:10034000C2F8AC30D1F8A830114A13F4806FF9D05C
:100350000321AA235520C2F8A010C2F8AC301146E0
:10036000C2F8AC00D1F8A800094A10F4407FF9D0D7
:100370000949002043F23A03C2F8A801C2F8AC01CF
:10038000C2F8C410C2F8C801136030BC704700BF87
:1003900000C00F4063000500DE87280430B5254DFE
:1003A000254BD5F8C41083B041F00074C5F8C440A3
:1003B000D5F8C420032042F01001C5F8C4101A6813
:1003C000002442F002051D60196821F001021A6044
:1003D0001D6845F0080119601A6822F004051D60C7
:1003E000196841F080421A601D6825F000411960CB
:1003F0005A6842F001055D605968104D21F0020213
:100400005A6000F0AFF90822012328604FF416511A
:10041000009400F089F9012000F0A4F9084D4FF490
:100420001641286008220123009400F07DF903B0F2
:1004300030BD00BF00C00F4000C002400C000010E3
:1004400014000010164A10B5D2F8C410154B41F430
:100450000044C2F8C4401968134841F434021A60D9
:100460005969124C21F480225A61596921F4801291
:100470005A61596921F400125A61596921F4000244
:100480005A6100F079F900F007FA2060084800F09E
:1004900073F900F001FA2060FFF780FF002010BD23
:1004A00000C00F4020C00920005A62021000001056
:1004B00000B4C404024B0146186800F003B800BF42
:1004C00014000010436913F0200FFBD00160704747
:1004D0000B7843B1426912F0200FFBD0036011F892
:1004E000013F002BF6D1704730B42A4A84B00DF199
:1004F000040C04460D46284B07CAACE803009C4296
:100500008CF8002029D018DD244B9C421BD003F529
:1005100080418C4214D104A94D19214B15F80C0CC3
:10052000D3F8AC11820442EA0101C3F8AC11D3F84C
:10053000AC010240C3F8AC2102E01A4884421ED04C
:1005400004B030BC70470DF1100C6544144B15F825
:100550000C2CD3F8AC111204E5E704A94D19104B8B
:1005600015F80C0CD3F8A811020242EA0101C3F8F5
:10057000A811D3F8A8010240C3F8A821E0E70DF1C3
:10058000100C6544064B15F80C2CD3F8A8119201F9
:10059000EBE700BF180F0000000001400080094099
:1005A00000C00F4000C000402DE9F047044682B073
:1005B0000F46002853D000F06FF9554E554B80463A
:1005C00030689C42019000F09C804BDD524B9C4275
:1005D0005DD003F5804294425FD0002302A800EB77
:1005E000030E1EF804CC3F01B8FBFCF3BB422BD238
:1005F000D6F80090474DDFF820A1AC42CDF804902A
:1006000067D050DC454B9C4235D000230DF1080EDD
:100610000EEB030C1CF8041C012920D049082046CD
:10062000FFF762FF3268AC4201925ED046DC3B4885
:10063000844226D0002302A901EB030E1EF804CC4D
:10064000B8FBFCF3BB42D8D3E268B3FBF7F342F04C
:100650008001E1602360E06820F08002E26002B087
:10066000BDE8F0872D498C42B7D12D48D0F8A8318C
:10067000C3F38113B2E72A48D0F8A821C2F381134B
:10068000C4E7274AD2F8A811C1F38113D3E724485D
:10069000D0F8AC31C3F30143A0E7214AD2F8AC1142
:1006A000C1F381439AE7544519D01E498C42ACD11D
:1006B0001B49D1F8AC31C3F38143A7E754451AD0A5
:1006C000184B9C42B6D1164BD3F8AC01C0F3814312
:1006D000B1E71349D1F8A831C3F3012396E71048D5
:1006E000D0F8AC21C2F3014390E70D4BD3F8A80139
:1006F000C0F301239FE70A4AD2F8AC11C1F30143CA
:1007000099E7074AD2F8A811C1F3012366E700BFB1
:10071000240F0000000001400080094000C000409C
:1007200000C00F4000C0094030B4092A9DF80840BD
:100730000ED8013BDDB2053A012D0ED90023072C5E
:100740000ED900259C186419C46030BCFFF72CBF7B
:10075000013BDDB20322012DF0D89B00072CF0D81D
:10076000E500EFE703289ABF024B53F82000002072
:10077000704700BF080F0000F0B4404D3F4CD5F863
:100780000C31D4F80C1113F0030F08BF3C4B3B4E57
:1007900001F003070CBF1A6842F21072D6F80C5130
:1007A000012F08BF374F05F0030308BF3A68022B3B
:1007B00008BF354B314908BF1A68344BB3FBF0F41E
:1007C000601EC1F804015000012218E0B4FBF0F1F2
:1007D000CF1F0132B7F5FC7F144622D9B5FBF0F1EB
:1007E000CD1F0132B5F5FC7F1BD9B6FBF0F1CD1F53
:1007F000A21CB5F5FC7F14D9E21C212A3BD0234969
:10080000234F244E5C18B3FBF0F1DD199E19CF1F66
:1008100003F18E4303F5060CB7F5FC7F0CF50C4392
:10082000D4D8541E154B220401398918AA24552006
:100830000122C3F88410C3F88C401946C3F88C0019
:10084000C3F88020C3F88C40C3F88C00D1F888002E
:100850000A4A10F0806FF9D00321AA205523C2F86C
:100860008010C2F88C001146C2F88C30D1F8882074
:1008700012F0407FFAD0F0BC704700BF00C00F40BC
:1008800004000010000000100800001000A3E11197
:100890000046C32300E9A4351C4A30B4D2F8845082
:1008A000D2F88440D2F80411D2F80C3113F0030FBF
:1008B00004BF174B1868154BD3F80C2102F0030C3A
:1008C000124ABCF1010FD2F80C2108BF114B02F003
:1008D000030C08BF1868BCF1020F04BF0E4B186868
:1008E0000A4BD3F8802012F0020F0CD0AA04930C0C
:1008F0005A1C5300C4F307444A1C00FB03F004FBDA
:100900000221B0FBF1F030BC704700BF00C00F40C7
:100910000400001000000010080000100FB42DE9C2
:10092000F04784B00CAB53F8045BDFF8FC803D4F1C
:1009300000240393287840B125280CD00135FFF717
:10094000B9FD287801340028F6D1204604B0BDE86E
:10095000F04704B070476878013525285DD0253808
:10096000532855D8DFE810F09C025400540054007E
:1009700054005400540054005400540054005400D7
:1009800054005400540054005400540054005400C7
:1009900054005400540054005400540054005400B7
:1009A00054005400540054005400540054005400A7
:1009B0005400540054005400540054005400540097
:1009C00054005400540054005400540054005C017E
:1009D0005400540054005400540054005400540077
:1009E0005400540054016200540054005400540058
:1009F0005400540054005400540054005400540057
:100A00005400540054005400540054005400FB019E
:100A100003980135021D03928CE7FFF74BFD01356A
:100A2000013487E767666666280F0000039BEC4683
:100A3000D3F8009098E80700ACE8030000200433E6
:100A400081456E4603938CF800208DF80900C0F2B2
:100A50002C82B9F1000F40F3D98087FB09204FEABF
:100A6000E971C1EBA00303EB830EA9EB4E0A0AF177
:100A700030098DF80090002B00F0208287FB03C91D
:100A8000DA17C2EBA90202EB820CA3EB4C03303362
:100A90008DF80130002A00F00E8287FB023ED0174D
:100AA000C0EBAE0303EB830AA2EB4A0130318DF8B1
:100AB0000210002B00F0048287FB03C9DA17C2EB97
:100AC000A90202EB820CA3EB4C0330338DF8033008
:100AD000002A00F0FB8187FB023ED017C0EBAE037B
:100AE00003EB830AA2EB4A0130318DF80410002B8E
:100AF00000F0E98187FB03C9DA17C2EBA90202EB18
:100B0000820CA3EB4C0330338DF80530002A00F043
:100B1000E08187FB023ED017C0EBAE0303EB830AF4
:100B2000A2EB4A0130318DF80610002B00F0D7817E
:100B300087FB03C9DA17C2EBA90202EB820CA3EB15
:100B40004C0330338DF80730002A00F0C58187FB55
:100B5000023ED017C0EBAE0303EB830AA2EB4A01BF
:100B600030318DF80810002B00F0BC8187FB03C9E1
:100B7000D817C0EBA90202EB820CA3EB4C03303375
:100B80008DF809304FF0090A16F80A00FFF792FCB9
:100B9000BAF1000F0AF003030AF1FF3936DDD3B1D1
:100BA000012B0DD0022B05D016F80900FFF782FCAF
:100BB00009F1FF3916F80900FFF77CFC09F1FF394C
:100BC00016F8090009F1FF39FFF774FC09F1010C6F
:100BD000BCF1000F1ADD16F8090009F1FF3AFFF722
:100BE00069FC16F80A00A9F1020AFFF763FC16F87F
:100BF0000A00FFF75FFCA9F10303F05CA9F1040907
:100C0000FFF758FC09F101010029E4DC013591E608
:100C1000039A0135111D10780391FFF74BFC89E60B
:100C200003996E460A68081D02F00F03092B88BF5E
:100C30000733039098E8030086E80300111101F0E0
:100C40000F003033092888BF07300A118DF80030B3
:100C500002F00F033030092B88BF073311118DF8D4
:100C6000010001F00F00092888BF0730091101F0C9
:100C70000F023030092A88BF073203F130090B1107
:100C80008DF8030003F00F00092888BF07301B11FF
:100C900002F1300C03F00F02092A00F1300188BF85
:100CA0000732C3F303103032092888BF07303030D1
:100CB0008DF802908DF804C08DF805108DF806208F
:100CC0008DF80700082300E04B4603F1FF3916F8C2
:100CD00009003028F8D0002B98DDFFF7EBFBB9F1C5
:100CE000000F09F0030309F1FF3A8FDDD3B1012BA7
:100CF0000DD0022B05D016F80A00FFF7DBFB0AF136
:100D0000FF3A16F80A00FFF7D5FB0AF1FF3A16F88A
:100D10000A000AF1FF3AFFF7CDFB0AF101010029B1
:100D20007FF774AF16F80A000AF1FF39FFF7C2FB2C
:100D300016F80900AAF10209FFF7BCFB16F8090032
:100D4000FFF7B8FBAAF10303F05CAAF1040AFFF76E
:100D5000B1FB0AF1010CBCF1000FE3DC56E703998B
:100D60006E460A68081D02F00F03092B88BF27335F
:100D7000039098E8030086E80300111101F00F00CA
:100D80003033092888BF27300A118DF8003002F06F
:100D90000F033030092B88BF273311118DF8010064
:100DA00001F00F00092888BF2730091101F00F0258
:100DB0003030092A88BF273203F1300C0B118DF82F
:100DC000030003F00F00092888BF27301B1102F130
:100DD000300903F00F02092A88BF27328DF802C0BC
:100DE00000F1300CC3F303103032092888BF2730DC
:100DF00030308DF804908DF805C08DF806208DF800
:100E00000700082300E04B4603F1FF3916F80900FC
:100E10003028F8D0002B7FF7F9AEFFF74BFBB9F184
:100E2000000F09F0030309F1FF3A7FF7EFAED3B1EA
:100E3000012B0DD0022B05D016F80A00FFF73AFB64
:100E40000AF1FF3A16F80A00FFF734FB0AF1FF3AFD
:100E500016F80A000AF1FF3AFFF72CFB0AF101032A
:100E6000002B7FF7D3AE16F80A000AF1FF39FFF71F
:100E700021FB16F80900AAF10209FFF71BFB16F87F
:100E80000900FFF717FBAAF10303F05CAAF1040ABB
:100E9000FFF710FB0AF1010CBCF1000FE3DCB5E633
:100EA00025200135FFF706FB44E52D20C9F1000997
:100EB000FFF700FBCDE54FF0010A65E69A4663E6D1
:100EC0004FF0020A60E64FF0040A5DE64FF0030AB5
:100ED0005AE64FF0050A57E64FF0070A54E64FF07E
:100EE000060A51E64FF0080A4EE600BF48656C6CF2
:100EF0006F20576F726C640A0D0000007465737484
:100F0000202564200A0D000000C0004000000140C0
:100F10000080094000C009400101020200000000F9
:100F200003000000040102082020202020202020AF
:040F300000000000BD
:0C0F3400001BB70000093D000080000019
:00000001FF
